:100000000C942A000C9447000C9447000C94470071
:100010000C9447000C9447000C9476010C949A01C0
:100020000C9447000C9447000C9447000C94470034
:100030000C9447000C9447000C9447000C94470024
:100040000C9447000C9447000C9447000C94470014
:100050000C94470011241FBECFE5D4E0DEBFCDBF16
:1000600010E0A0E6B0E0E6E1F4E002C005900D92F9
:10007000A437B107D9F710E0A4E7B0E001C01D92A2
:10008000AA37B107E1F70E94B7000C9409020C945B
:10009000000086958695813318F0E0E4E81B04C0E3
:1000A000813240F08052E82FF0E0E05AFF4F80812B
:1000B00081950895813138F0E0E2E81BF0E0E05AE4
:1000C000FF4F80810895E82FF0E0E05AFF4F8081D4
:1000D0000895809171009091720041E09C01220F7F
:1000E000331F8227932796FD02C0C90102C0C901B0
:1000F00081604F5F483091F7809371009093720058
:1001000008950F931F93CF93DF938C01C0E0D0E04D
:1001100005C081E090E00E94D8012196C017D10768
:10012000C0F3DF91CF911F910F9108950F931F930B
:100130008B01880F991F880F991F0E940401C80125
:10014000880F991F880F991F0E943D011F910F91E1
:1001500008950E94BE010E94E20080E090E00E94AB
:10016000040180E090E00E943D01789408950E948F
:10017000A90080ED97E00E94810068EC70E088ECB7
:1001800090E00E9496000E94C201882321F40E9400
:10019000CD018823A1F068E37FEF88E39FEF0E9401
:1001A00096008CED95E00E9481006CE07EEF84EF7C
:1001B00091E00E9496008CE291E00E9481008AE02A
:1001C00090E0D9CF8091790082608093790082B3EA
:1001D000806F82BB81B3806F81BB82EF8FBD81E076
:1001E0008EBD89B789BF08958FB7F89410927600B5
:1001F0001092750010927800109277001BBC1ABC08
:1002000019BC18BC8FBF089562E070E00E94E20143
:10021000CB0122E060307207D4F42EEF6130720718
:100220001CF481E09EEF02C077FF13C02227332722
:10023000281B390B3093760020937500969B04C0E1
:1002400080917400827011C03BBD2ABD08958FEF6C
:1002500091E09093760080937500969B03C09BBDC0
:100260008ABD0895809174008160809374001BBCE6
:100270001ABC89B7806189BF089562E070E00E946E
:10028000E201CB0122E060307207D4F42EEF61303E
:1002900072071CF481E09EEF02C077FF13C0222793
:1002A0003327281B390B3093780020937700979BD6
:1002B00003C039BD28BD08958091740082600BC0D1
:1002C0008FEF91E09093780080937700979B0BC01D
:1002D0008091740081708093740019BC18BC89B738
:1002E000886089BF089599BD88BD08951F920F92B7
:1002F0000FB60F9211248F939F93859B14C092B3D6
:100300008091740080FD02C080E001C080E49F7B8A
:10031000892B82BB80917500909176009BBD8ABD30
:1003200089B78F7E89BF9F918F910F900FBE0F90DD
:100330001F9018951F920F920FB60F9211248F9352
:100340009F93849B14C092B38091740081FD02C07E
:1003500080E001C080E89F77892B82BB8091770085
:100360009091780099BD88BD89B7877F89BF9F919B
:100370008F910F900FBE0F901F90189585B3806FCF
:1003800085BB089593B39073903111F48FEF089566
:1003900080E0903209F481E0089593B3907C90342A
:1003A00011F48FEF089580E0903809F481E008950A
:1003B00026EA3EE004C0F9013197F1F70197009772
:1003C000D1F7089597FB092E07260AD077FD04D0B0
:1003D0000CD006D000201AF4709561957F4F0895D7
:1003E000F6F7909581959F4F0895AA1BBB1B51E18D
:1003F00007C0AA1FBB1FA617B70710F0A61BB70B95
:10040000881F991F5A95A9F780959095BC01CD0139
:060410000895F894FFCFEF
:10041600000C1925313C47515A626A70757A7D7E07
:040426007FAA0000A9
:00000001FF
